:020000040000FA
:020000000728CF
:0800080015204C2809008316A5
:10001000013086000130850083128B170B164C28A7
:10002000051C102805181228080005128601080072
:10003000152005166E3086000800152005167E3046
:1000400086000800152005160630860008001520D9
:1000500005167C3086000800152005166C308600D9
:1000600008001520663086000800152005164E3061
:1000700086000800152005165A3086000800152055
:10008000063086000800152005163E308600080060
:10009000152080308600080083120B108B108B1700
:1000A0001020182010201D20102022201020272092
:1000B00010202C20102031201020352010203A2034
:0E00C00010203F2010204320102048206528EB
:02400E00F13F80
:00000001FF
